:1000000000A00120110500008D0500008F050000F3
:100010009105000093050000950500000000000018
:100020000000000000000000000000009705000034
:1000300099050000000000009B0500006D280000ED
:100040009F050000A3050000A7050000AB05000008
:10005000AF050000B3050000B7050000BB050000B8
:10006000BF050000C3050000C7050000CB05000068
:10007000CF050000D3050000D7050000DB05000018
:10008000DF050000E3050000E7050000EB050000C8
:10009000EF050000F3050000F7050000FB05000078
:1000A000FF05000003060000070600000B06000025
:1000B0000F06000013060000890500001706000067
:1000C0001B0600001F060000230600002706000094
:1000D000890500002B0600002F06000033060000F3
:1000E000370600003B060000890500003F060000BF
:1000F00043060000470600004B0600004F060000C4
:100100008905000053060000570600005B0600004A
:100110005F06000063060000670600006B06000033
:100120006F06000073060000770600007B060000E3
:100130007F06000083060000870600008B06000093
:100140008F06000093060000970600009B06000043
:100150009F060000A3060000A7060000AB060000F3
:10016000AF060000B3060000B7060000BB060000A3
:10017000BF060000C3060000C7060000CB06000053
:10018000CF060000D3060000D7060000DB06000003
:10019000DF060000E3060000E7060000EB060000B3
:1001A000EF060000F3060000F7060000FB06000063
:1001B000FF06000003070000070700000B07000010
:1001C0000F07000013070000170700001B070000BF
:1001D0001F07000023070000270700002B0700006F
:1001E0002F07000033070000370700003B0700001F
:1001F0003F07000043070000470700004B070000CF
:100200004F07000053070000570700005B0700007E
:100210005F07000063070000670700006B0700002E
:100220006F07000073070000770700007B070000DE
:100230007F07000083070000870700008905000092
:100240008905000089050000890500008905000076
:100250008905000089050000890500008905000066
:100260008905000089050000890500008905000056
:100270008905000089050000890500008905000046
:100280008905000089050000890500008905000036
:100290008905000089050000890500008905000026
:1002A00089050000890500008B0700008F0700000A
:1002B00093070000970700009B0700009F070000BE
:1002C000A3070000A7070000AB070000AF0700006E
:1002D000B3070000B7070000BB070000BF0700001E
:1002E000C3070000C7070000CB070000CF070000CE
:1002F000D3070000D7070000DB07000089050000D6
:10030000DF070000E3070000E7070000EB0700003D
:10031000EF070000F3070000F7070000FB070000ED
:10032000FF07000003080000070800000B0800009A
:100330000F08000013080000170800001B08000049
:100340001F08000023080000270800002B080000F9
:100350002F08000033080000370800003B080000A9
:100360003F08000043080000470800004B08000059
:040370004F08000032
:10040000FFFFFFFFFFFFFFFFFFFFFFFFFE7FFFFF7D
:100410004730305F50733036365F535750422D5659
:10042000462D312E303030342E30300000000000A8
:100430004A756C2020312032303234000000000038
:1004400030313A34363A313000000000000000000C
:10045000303030303030303030303030000000005C
:10046000000000000000000000000000000000008C
:10047000000000000000000000000000000000007C
:1004800000000000000000000C0000002000000040
:10049000000000000000000000000000000000005C
:1004A000000000000000000000000000000000004C
:1004B000000000000000000000000000000000003C
:1004C000000000000000000000000000000000002C
:1004D000000000000000000000000000000000001C
:1004E000000000000000000000000000000000000C
:1004F00000000000000000000000000000000000FC
:1005000000000000000000000000000000000000EB
:1005100072B61348134901600A6882F308881249C9
:10052000124A521A013A05DD0020042308601944DA
:10053000043AFBDA0E490F4A0F4B9A42BEBF51F8FC
:10054000040B42F8040BF8E70C490D4A00209142D5
:10055000BCBF41F8040BFAE762B60A480047000046
:1005600008ED00E00000000000100020FF9F0120C7
:10057000F82F000000100020241000202810002078
:1005800004130020010E0000FFF7FEBFFEE7FEE7A8
:10059000FEE7FEE7FEE7FEE7FEE7FEE7FEE7AD4823
:1005A0000047AD480047AD480047AD480047AD485B
:1005B0000047AD480047AD480047AD480047AD484B
:1005C0000047AD480047AD480047AD480047AD483B
:1005D0000047AD480047AD480047AD480047AD482B
:1008500000470000890500008905000089050000A7
:100860008905000089050000890500008905000050
:100870008905000089050000890500008905000040
:100880008905000089050000890500008905000030
:1008900089050000890500000514000029140000E6
:1008A00089050000750E000089050000890500001B
:1008B00089050000890500004D2600005326000030
:1008C00059260000652600005F2600006B26000008
:1008D0007126000077260000832600007D26000098
:1008E000892600008F26000095260000A126000022
:1008F0009B260000A7260000AD260000B3260000BE
:10090000BF260000B9260000890500008905000007
:10091000890500008905000089050000890500009F
:10092000D11E0000DF1E0000ED1E0000FB1E0000B7
:10093000091F0000171F0000251F0000331F0000C3
:10094000411F00004F1F00005D1F00006B1F0000D3
:10095000791F0000871F0000951F0000A31F0000E3
:10096000B11F0000BF1F0000CD1F0000DB1F0000F3
:10097000E91F0000F71F0000052000001320000001
:10098000212000002F2000003D2000004B2000000F
:10099000592000006720000075200000832000001F
:1009A000912000009F200000AD200000BB2000002F
:1009B000C9200000D7200000E5200000F32000003F
:1009C000012100000F2100001D2100002B2100004B
:1009D000392100004721000055210000632100005B
:1009E000712100007F2100008D2100009B2100006B
:1009F000A9210000B7210000C5210000D32100007B
:100A0000E1210000EF210000FD2100000B22000089
:100A10001922000027220000352200004322000096
:100A2000512200005F2200006D2200007B220000A6
:100A30008922000097220000A5220000B3220000B6
:100A4000890500008905000089050000890500006E
:100A5000890500008905000089050000890500005E
:100A6000890500008905000089050000890500004E
:100A7000890500008905000089050000890500003E
:100A8000890500008905000089050000890500002E
:100A9000890500008D1500009315000099150000D0
:100AA0009F150000A51500008905000089050000BC
:100AB00089050000890500008905000089050000FE
:100AC00089050000890500008905000089050000EE
:100AD000210F00008905000089050000890500003C
:100AE00089050000890500008905000089050000CE
:100AF00089050000892300008F230000890500007C
:100B0000890500008905000053B94AB9002908BFCA
:100B100000281CBF4FF0FF314FF0FF3000F06EB9DE
:100B2000ADF1080C6DE904CE00F006F8DDF804E044
:100B3000DDE9022304B070472DE9F047089D044623
:100B40008C46002B40F083808A42174647D9B2FA80
:100B500082F242B1C2F1200024FA00F091409740A5
:100B600040EA010C94404FEA1748230CBCFBF8F60E
:100B70001FFA87FE08FB16C143EA014306FB0EF18C
:100B8000994209D9FB1806F1FF3080F0198199428A
:100B900040F21681023E3B445B1AA4B2B3FBF8F06C
:100BA00008FB103344EA034400FB0EFEA64509D9B6
:100BB0003C1900F1FF3380F00581A64540F2028127
:100BC00002383C4440EA0640A4EB0E0400261DB166
:100BD000D4400023C5E900433146BDE8F08702B99F
:100BE000FFDEB2FA82F2002A50D1CB1B4FEA174E39
:100BF0001FFA87F80126B3FBFEFC210C0EFB1C3309
:100C000041EA034108FB0CF38B4207D979180CF138
:100C1000FF3002D28B4200F2E9808446C91AA3B2A7
:100C2000B1FBFEF00EFB101143EA014408FB00F893
:100C3000A04507D93C1900F1FF3302D2A04500F2CC
:100C4000D9801846A4EB080440EA0C40BFE78B4269
:100C500009D9002D00F0B1800026C5E90001304619
:100C60003146BDE8F087B3FA83F6002E4AD18B42B5
:100C700002D3824200F2B880841A61EB03010120A2
:100C80008C46002DA8D0C5E9004CA5E7C2F1200391
:100C900020FA03F6974001FA02F04FEA174ED940C6
:100CA0003043030CB1FBFEF61FFA87F80EFB16115A
:100CB00043EA014306FB08F1994204FA02F409D918
:100CC000FB1806F1FF3C80F08D80994240F28A804B
:100CD000023E3B445B1A81B2B3FBFEF00EFB1033C5
:100CE00041EA034100FB08F38B4207D9791800F170
:100CF000FF3C73D28B4271D902383944CB1A40EA97
:100D0000064678E7C6F1200C03FA06F422FA0CF343
:100D10001C4320FA0CF701FA06F34FEA144E21FAAD
:100D20000CF11F433B0CB1FBFEF91FFA84F80EFBDC
:100D3000191143EA014109FB08FA8A4502FA06F251
:100D400000FA06F308D9611809F1FF3048D28A4544
:100D500046D9A9F102092144A1EB0A01BFB2B1FBB6
:100D6000FEF00EFB101147EA014700FB08F8B845FA
:100D700007D9E71900F1FF312ED2B8452CD9023836
:100D8000274440EA0940A7EB0807A0FB02894F452A
:100D9000C64649461AD317D05DB1B3EB0E0267EBD6
:100DA000010707FA0CFCF2404CEA0202F740C5E9E1
:100DB000002700263146BDE8F0872E4628460BE77F
:100DC0000646E9E61846FDE64345E5D2B8EB020ED5
:100DD00069EB04010138DFE70846D2E760468DE79A
:100DE0008146B9E7664675E730464AE7ACF1020C42
:100DF000394413E702383C4424E700BF704700BF82
:100E000008B501F05DFE002008BD000082B000239F
:100E1000084A01939368DB0102D5002002B07047B5
:100E2000019BB3F5801F03D2019B01330193F1E7CE
:100E30000120F3E70020054072B607B403480449D7
:100E4000044A0160026007BC62B670471420054086
:100E5000C4A1D9B00F3B1E1A08B5FFF7EDFF044B34
:100E60009A686FF300029A60BDE80840FFF7CEBFB2
:100E70000020054008B5034B1B6803B19847BFF33A
:100E80004F8F08BD28100020124BDA6A002ABCBF21
:100E90004FF0B642DA62DA6A417861F31242DA62FE
:100EA000DA6A017861F30102DA62DA6A017961F3E0
:100EB0000F22DA62DA6A417A61F30412DA62DA6ADC
:100EC000017A61F34512DA62DA6A42F00042DA62CC
:100ED000704700BF00400640074B5A69002ABCBF5C
:100EE0004FF0B6425A615A696FF349225A615A6902
:100EF00042F000425A61704700400640074BDA69F1
:100F0000002ABCBF4FF0B642DA61DA696FF34922BA
:100F1000DA61DA6942F00042DA6170470040064067
:100F200008B51A4B5A69510311D55A69002ABCBF3A
:100F30004FF0B6425A615A6942F480225A615A69A6
:100F400042F000425A61124B1B68CBB198470F4BDD
:100F5000DA69520311D5DA69002ABCBF4FF0B642F4
:100F6000DA61DA6942F48022DA61DA6942F0004239
:100F7000DA61074B5B6833B19847BFF34F8F08BD09
:100F8000FFF7AAFFE3E7FFF7B9FFF6E700400640E7
:100F90002C1000208C283CD877280CD8542832D824
:100FA000372819D8142828D803281FD93E4B0122E6
:100FB0008240134019E0A0F17803142B16D8DFE823
:100FC00003F0351515153515151515151515154895
:100FD0005A67351515153500A0F13803DAB201232B
:100FE000934003F0113323F48833FBB97047012297
:100FF00002FA03F313F0113F17E0A0F11803DBB27C
:101000001C2BF4D97047A0F15803DBB21C2BEED98E
:101010007047A0280AD000F15003DBB2102BE5D8AE
:10102000012202FA03F3214A1342DFD0204B800849
:1010300053F820301A68002ABCBF4FF0B6421A603D
:101040001A6861F30B221A601A6842F000421A60B3
:101050007047184BDA68002ABCBF4FF0B642DA601E
:10106000DA6822F4706242EA0121D960DA6842F05B
:101070000042DA60BAE70F4BDA68002ABCBF4FF0D3
:10108000B642DA60DA6822F0F00242EA0111ECE7D7
:10109000084BDA68002ABCBF4FF0B642DA60DA6863
:1010A00022F00F021143E0E71011110011110100AD
:1010B000B42C00000040064082084D4B82B053F82B
:1010C00022307C284FF000028DF8072053D85F288B
:1010D0000AD83C283CD81F2822D8021F182A2BD90E
:1010E00001238DF8073017E06038C0B2012202FA00
:1010F00000F010F0113FF3D01A68002ABCBF4FF087
:10110000B6421A60012956D11A6861F306121A60B4
:101110001A6842F000421A609DF8070002B070475A
:1011200020380122C0B202FA00F0324A10421BD12C
:1011300040F211121042DEE7012202FA00F000F044
:10114000113222F01102002AD6D110F0100F23E044
:101150004038C0B21C28C3D8012202FA00F0254A48
:101160001042C9D1C207BBD51A68002ABCBF4FF0D4
:10117000B6421A6021E0A0282BD004D800F0FB0072
:101180008828ADD109E05030C0B21028A8D801227B
:1011900002FA00F0184A1042A2D01A68002ABCBF16
:1011A0004FF0B6421A600129AED00229ACD0032913
:1011B000AAD0042906E00229A6D00329A4D0042934
:1011C000A2D00529A0D000299ED001228DF80720A9
:1011D0009EE71A68002ABCBF4FF0B6421A60032986
:1011E00092D0042990D005298ED00629EAE700BFC5
:1011F000B42C0000001011111111010082B0002365
:101200000138019304283FD8DFE800F033271B0F93
:101210000300204A2049936ADB032FD4019B8B42B1
:1012200032D8019B01330193F5E71A4A1A495369F1
:10123000D80323D4019B8B4226D8019B0133019311
:10124000F5E7144A1449D369D80317D4019B8B429C
:101250001AD8019B01330193F5E7104A104913682E
:101260009B050BD4019B8B420ED8019B013301934C
:10127000F5E70C4A084953685B0702D5002002B025
:101280007047019B8B4201D90120F8E7019B013394
:101290000193F0E700400640A0860100009007405F
:1012A000404B4C0000D0074010B5154CA36A002BF2
:1012B000BCBF4FF0B643A362A36A43F40073A362BA
:1012C000A36A60F34103A362A36A43F00103A3622C
:1012D000A36A43F00043A3620520FFF78FFF70B9B4
:1012E0004FF0B643A362A36A43F00073A362A36AFC
:1012F00060F34923A362A36A43F00043A36210BDD5
:101300000040064010B4174B9C69002CBCBF4FF046
:10131000B6449C619C6960F382049C61986962F3A5
:10132000000098619A6942F002029A619A6942F05B
:1013300000429A615A69002ABCBF4FF0B6425A6116
:10134000084B5A6961F341025A615A6942F001023D
:101350005A615A6942F000425A615DF8044B042018
:10136000FFF74CBF00400640012808B517D1032005
:10137000FFF744FF08B1012008BD1D4BDA68002AC1
:10138000BCBF4FF0B642DA60DA6822F4E02242F4E1
:101390008032DA60DA6842F00042DA60ECE7022874
:1013A00011D10420FFF72AFF0028E4D1104BDA689E
:1013B000002ABCBF4FF0B642DA60DA6822F4E022BD
:1013C00042F40032E5E70328D5D10520FFF716FFE8
:1013D0000028D0D1064BDA68002ABCBF4FF0B642D5
:1013E000DA60DA6822F4E02242F44032D1E700BF4A
:1013F00000400640024B9A6860F303029A6070470F
:101400000000024008B5064B5A686FF3C7125A60D5
:10141000044B1B6803B19847BFF34F8F08BD00BF53
:101420000000024034100020104B10B51C685A68B0
:10143000144004F440321A60E20303D50C4A5268A7
:101440004AB19047A30303D5094B9B6843B1984722
:10145000BFF34F8F10BD5A6822F480325A60F1E713
:10146000024A536823F400335360F1E7000002405E
:10147000341000200B4B800853F820301A68002AE3
:10148000BCBF4FF0B6421A601A686FF355521A602B
:101490001A6842F400121A601A6842F000421A6098
:1014A000704700BF882D00000B4B8008012153F8C6
:1014B00020301A68002ABCBF4FF0B6421A601A6882
:1014C00061F301021A601A6842F400121A601A6885
:1014D00042F000421A607047882D00000B4B8008D4
:1014E00053F820301A68002ABCBF4FF0B6421A6089
:1014F0001A686FF301021A601A686FF355521A6086
:101500001A6842F000421A60704700BF882D000040
:101510002DE9F84F1A4BDFF870A053F82050194B03
:10152000D5F8907053F82090064600244FF0B64B43
:101530004FF0010827FA04F3DB0705D5DAF800209D
:1015400072B1E1B23046904708FA04F301343B40EF
:10155000202CC5F89030EDD1BFF34F8FBDE8F88F48
:10156000231D49F823B055F8231062F3134145F8C1
:10157000231055F8232042F4004245F82320E3E7E6
:10158000702E0000842E0000401000200020FFF785
:10159000BFBF0120FFF7BCBF0220FFF7B9BF032088
:1015A000FFF7B6BF0420FFF7B3BF00000E4B0431B6
:1015B00053F8203010B553F82140240441BF0B4CA0
:1015C00054F820004FF0B64440F8214053F8210071
:1015D00062F30A2043F8210053F8212042F400422C
:1015E00043F8212010BD00BF702E0000842E0000A3
:1015F000064B10B553F8204001206369884023EA68
:10160000000302FA01F10B43636110BD5C2E000080
:10161000194B82B053F820301848002101911A6804
:1016200042F080421A601A6842F080521A601A68CA
:101630008A42BEBF1A6861F3DF721A600146019ADE
:10164000824205D8019A013201921A681201F6D538
:10165000019A8A4204D800220192019A8A4202D950
:10166000012002B07047019A013201921A68D2013A
:10167000F3D50020F5E700BF142F00003F4B4C00CE
:101680000F4B82B053F8203000220192196862F3A8
:101690001C711960196862F39E71196042F20F7132
:1016A000019A8A4201D9012007E0019A0132019290
:1016B0001A68C2F30060D201F2D402B0704700BFD2
:1016C000142F00002D4B2DE9F04753F820A02C4B90
:1016D000DAF8006053F82040DFF8A890236BA26A84
:1016E00006F07F06013603EA0208102E4FF04C0781
:1016F0001FFA88F828BF10260025474328FA05F36B
:10170000DA070FD5DAF800309B0020D5072D1ED858
:10171000052D11D109EB0703DB6A43B1984701237B
:10172000AB4023630135AE42E8D1BDE8F087A36A40
:1017300023F02003A362F2E7062D14D109EB07037F
:101740001B6B002BEAD1A36A23F04003F2E759F8A0
:10175000073013B128469847E1E7A36A0122AA405F
:1017600023EA0203E6E7072DD9D109EB07035B6BF8
:10177000002BD3D1A36A23F08003DBE7142F0000F2
:101780002C2F0000741000201D4B1E4A53F82030EF
:101790002DE9F04752F820901C68D9F83030D9F87C
:1017A0002820DFF864A004F07F04013403EA020873
:1017B0004FEA1848202C4FF04C074FEA084828BF42
:1017C000202410254743A54201D3BDE8F08728FA1D
:1017D00005F30126DB0706FA05F605D50AEB070334
:1017E0005B682BB128469847C9F830600135EAE7B5
:1017F000D9F8283023EA0603C9F82830F4E700BFF7
:10180000142F00002C2F0000741000201B4B1C4ACA
:1018100053F820302DE9F0471C6852F82060DFF8BB
:1018200064A0F76A736A04F07F0401341F40302C0F
:101830004FF04C09BFB228BF3024202509FB00F926
:10184000A54201D3BDE8F087A5F120034FF00108C0
:1018500008FA03F827FA03F3DB0705D50AEB0903B7
:101860009B6833B1284698470135C6F82C80EDB205
:10187000E6E7736A23EA08037362F5E7142F0000B2
:101880002C2F0000741000201C4B1D4A53F82030F0
:101890002DE9F04752F820701C68FD6A7B6ADFF87A
:1018A00064A004F07F0401341D402D0C402C4FF047
:1018B0004C094FEA054528BF4024302609FB00F9B2
:1018C000A64201D3BDE8F087A6F120034FF001083E
:1018D00008FA03F825FA03F3DB0705D50AEB090339
:1018E000DB682BB130469847C7F82C800136E7E714
:1018F0007B6A23EA08037B62F6E700BF142F00002F
:101900002C2F0000741000202DE9F74F0F46984946
:10191000DDF830A051F820509649DDF8349051F8A8
:10192000204029689846CB010646C1F3006B14D5C8
:10193000102F2FD8DFE817F04E004E00660066002B
:10194000870087009D00AF00AF00AF00BB00BB0069
:10195000BB00D400D4001900E3000192FFF758FE49
:10196000002840F04381019AE2E7B11FC9B2F2B901
:10197000A26A42EA0802A262636A012943EA0A03F0
:10198000636207D8E36E0E9A43EA0903E366A36E27
:101990001343A366BBF1000F40F02A813046FFF7E6
:1019A0006FFE003818BF012003B0BDE8F08FA26AB7
:1019B00022EA0803A362636A012923EA0A03636235
:1019C000E8D8E36E0E9A23EA0903E366A36E23EADE
:1019D0000203DEE7684B6948694D53F8271055F854
:1019E000275050F8263032B962682A4362600B43B0
:1019F00040F82630CEE7626822EA0502626023EAF8
:101A00000103F5E75C4B5D495D4853F827C051F889
:101A1000263050F827705AB9286840F40010286022
:101A200062683A43626043EA0C0341F82630B1E74A
:101A30002A686FF355522A60626822EA07026260E0
:101A400023EA0C03F1E74C4B4C494D4D53F827006A
:101A500055F8275051F8263022B9626B2A43626349
:101A60000343E2E7626B22EA0502626323EA0003B2
:101A7000DBE7424951F8263032B9226842F08062F1
:101A8000226043F00103D0E7226822F080622260E6
:101A900023F00103C9E73A4B53F827301AB9A26A79
:101AA0001343A36276E7A26A22EA0303F9E76B6BAA
:101AB00043F000536B63D5F8E03A6FF3DF73C5F87A
:101AC000E03A2F4B53F827302AB9D4F8E02A1343D1
:101AD000C4F8E03A5EE7D4F8E02A22EA0303F7E725
:101AE000274B53F827302AB9D4F8002B1343C4F8F6
:101AF000003B4FE7D4F8002B22EA0303F7E7B11FBE
:101B00001E48A36AC9B2002A3ED14FF0FF33A36238
:101B1000626A636201299FBFE26EE366A26EA366FA
:101B2000636843F44C436360636B43F04043636317
:101B30006B6B43F000536B63D5F8E03A6FF3DF73E0
:101B4000C5F8E03AD4F8E03A43F45023C4F8E03A58
:101B50002B6843F080632B602B6843F400132B60E9
:101B6000D4F8003B43F44033C4F8003B054B3FE757
:101B7000142F00002C2F0000982E00005C10002075
:101B8000D82E000007001B000023A362626A636274
:101B900001299FBFE26EE366A26EA366636823F429
:101BA0004C436360636B23F0404363636B6B43F0B0
:101BB00000536B63D5F8E03A6FF3DF73C5F8E03A92
:101BC000D4F8E03A23F45023C4F8E03A2B686FF3DA
:101BD0009A632B602B686FF355532B60D4F8003B4E
:101BE00023F44033C4F8003B002301E70120DBE687
:101BF0000020D9E61A4B53F820201A4B30B553F881
:101C00002030156A1D40184B2B4013626A0785B0BF
:101C1000044606D5154A4C2303FB00231B6963B118
:101C200098472B0319D5114A4C2303FB04231B6A45
:101C30005BB105B0BDE830401847029301930093B3
:101C400001221946FFF760FEEBE702930193009330
:101C5000012204212046FFF757FE05B030BD00BF2A
:101C60002C2F00005C1000200400080074100020DD
:101C70001FB50D4A52F820204FF4003111620B4A73
:101C80004C2101FB00239B691BB105B05DF804EBFF
:101C9000184702930193009301220221FFF734FEBB
:101CA00005B05DF804FB00BF2C2F0000741000206D
:101CB0001FB50D4A52F820204FF4803111620B4AB3
:101CC0004C2101FB0023DB691BB105B05DF804EB7F
:101CD000184702930193009301220321FFF714FE9A
:101CE00005B05DF804FB00BF2C2F0000741000202D
:101CF0000F4B53F8203030B50E4D196A45F82010BF
:101D0000022119620C494C2303FB001385B05B6967
:101D100004462BB19847002345F8243005B030BD68
:101D200001220293019300931146FFF7EDFDF2E7C4
:101D30002C2F00004410002074100020104B53F88A
:101D4000203030B50F4D196A45F820104FF480113E
:101D500019620D494C2303FB001385B05B6A0446EE
:101D60002BB19847002345F8243005B030BD0293CD
:101D70000193009301220521FFF7C6FDF2E700BFA2
:101D80002C2F000044100020741000201A4B53F830
:101D9000203030B5D3F8082BD3F8005B154005F49C
:101DA0004032C3F8082BEA0385B0044606D5134A2F
:101DB0004C2303FB00235B6C63B19847AB0319D53D
:101DC0000E4A4C2303FB04239B6C5BB105B0BDE8BA
:101DD0003040184702930193009301220D21FFF731
:101DE00093FDEBE702930193009301220E2120461D
:101DF000FFF78AFD05B030BD2C2F000074100020C5
:101E00001FB50B4A52F8201001220A6209494C24DE
:101E100004FB00139B6A1BB104B0BDE810401847D7
:101E20000293019300930621FFF76EFD04B010BDED
:101E30002C2F000074100020234B53F8203030B5B5
:101E4000D3F8FC2AD3F8E05A154005F450222903B0
:101E500085B00446C3F8FC2A06D51C4A4C2303FB74
:101E600000239B6BABB198476A0306D5174A4C23F6
:101E700003FB0423DB6BA3B19847EB0322D5134A82
:101E80004C2303FB04231B6CA3B105B0BDE8304019
:101E9000184702930193009301220A21FFF734FDB2
:101EA000E2E702930193009301220B212046FFF702
:101EB0002BFDE2E702930193009301220C212046BF
:101EC000FFF722FD05B030BD2C2F0000741000205C
:101ED00008B50020FFF78EFEBFF34F8F08BD08B591
:101EE0000020FFF7C5FEBFF34F8F08BD08B50020E7
:101EF000FFF7DEFEBFF34F8F08BD08B50020FFF7E8
:101F0000F7FEBFF34F8F08BD08B50020FFF716FF9F
:101F1000BFF34F8F08BD08B50020FFF737FFBFF3B1
:101F20004F8F08BD08B50020FFF76AFFBFF34F8F42
:101F300008BD08B50020FFF77FFFBFF34F8F08BD36
:101F400008B50020FFF7BEFBBFF34F8F08BD08B5F3
:101F50000020FFF719FCBFF34F8F08BD08B5002024
:101F6000FFF754FCBFF34F8F08BD08B50020FFF703
:101F70008BFCBFF34F8F08BD08B50120FFF73AFE79
:101F8000BFF34F8F08BD08B50120FFF771FEBFF307
:101F90004F8F08BD08B50120FFF78AFEBFF34F8FB2
:101FA00008BD08B50120FFF7A3FEBFF34F8F08BDA2
:101FB00008B50120FFF7C2FEBFF34F8F08BD08B57B
:101FC0000120FFF7E3FEBFF34F8F08BD08B50120E6
:101FD000FFF716FFBFF34F8F08BD08B50120FFF7CD
:101FE0002BFFBFF34F8F08BD08B50120FFF76AFB39
:101FF000BFF34F8F08BD08B50120FFF7C5FBBFF346
:102000004F8F08BD08B50120FFF700FCBFF34F8FCD
:1020100008BD08B50120FFF737FCBFF34F8F08BD9F
:1020200008B50220FFF7E6FDBFF34F8F08BD08B5E6
:102030000220FFF71DFEBFF34F8F08BD08B5022039
:10204000FFF736FEBFF34F8F08BD08B50220FFF73C
:102050004FFEBFF34F8F08BD08B50220FFF76EFE9D
:10206000BFF34F8F08BD08B50220FFF78FFEBFF307
:102070004F8F08BD08B50220FFF7C2FEBFF34F8F98
:1020800008BD08B50220FFF7D7FEBFF34F8F08BD8C
:1020900008B50220FFF716FBBFF34F8F08BD08B548
:1020A0000220FFF771FBBFF34F8F08BD08B5022078
:1020B000FFF7ACFBBFF34F8F08BD08B50220FFF759
:1020C000E3FBBFF34F8F08BD08B50320FFF792FD78
:1020D000BFF34F8F08BD08B50320FFF7C9FDBFF35D
:1020E0004F8F08BD08B50320FFF7E2FDBFF34F8F08
:1020F00008BD08B50320FFF7FBFDBFF34F8F08BDF8
:1021000008B50320FFF71AFEBFF34F8F08BD08B5CF
:102110000320FFF73BFEBFF34F8F08BD08B5032038
:10212000FFF76EFEBFF34F8F08BD08B50320FFF722
:1021300083FEBFF34F8F08BD08B50320FFF7C2FA37
:10214000BFF34F8F08BD08B50320FFF71DFBBFF39A
:102150004F8F08BD08B50320FFF758FBBFF34F8F23
:1021600008BD08B50320FFF78FFBBFF34F8F08BDF5
:1021700008B50420FFF73EFDBFF34F8F08BD08B53B
:102180000420FFF775FDBFF34F8F08BD08B504208D
:10219000FFF78EFDBFF34F8F08BD08B50420FFF792
:1021A000A7FDBFF34F8F08BD08B50420FFF7C6FD9C
:1021B000BFF34F8F08BD08B50420FFF7E7FDBFF35D
:1021C0004F8F08BD08B50420FFF71AFEBFF34F8FED
:1021D00008BD08B50420FFF72FFEBFF34F8F08BDE1
:1021E00008B50420FFF76EFABFF34F8F08BD08B59E
:1021F0000420FFF7C9FABFF34F8F08BD08B50420CC
:10220000FFF704FBBFF34F8F08BD08B50420FFF7AD
:102210003BFBBFF34F8F08BD08B50520FFF7EAFC75
:10222000BFF34F8F08BD08B50520FFF721FDBFF3B1
:102230004F8F08BD08B50520FFF73AFDBFF34F8F5C
:1022400008BD08B50520FFF753FDBFF34F8F08BD4C
:1022500008B50520FFF772FDBFF34F8F08BD08B525
:102260000520FFF793FDBFF34F8F08BD08B505208C
:10227000FFF7C6FDBFF34F8F08BD08B50520FFF778
:10228000DBFDBFF34F8F08BD08B50520FFF71AFA35
:10229000BFF34F8F08BD08B50520FFF775FABFF3F0
:1022A0004F8F08BD08B50520FFF7B0FABFF34F8F79
:1022B00008BD08B50520FFF7E7FABFF34F8F08BD4B
:1022C0002D4B2DE9F04153F820502C4B53F8207042
:1022D0002B4BFE6853F820301E4026F00103FB60B4
:1022E000F307044607D51423264A4343D35843B380
:1022F00098470123FB60B00706D5224A142303FB4D
:1023000004235B6813B39847710706D51D4A14234D
:1023100003FB04239B68F3B19847320706D5194A9B
:10232000142303FB0423DB68D3B19847B30520D5FE
:102330001448142303FB04042369B3B1BDE8F0413E
:1023400018472A6963F300022A61D2E72A6963F316
:1023500041022A61D8E72A6963F382022A61DCE735
:102360002A6963F3C3022A61E0E72A6963F345122D
:102370002A61BDE8F08100BF442F00004C2F00000F
:102380003C120020441200200020FFF799BF0120DA
:10239000FFF796BF1A4B53F8203088789A680228C6
:1023A0001DBF6FF304129A605A6942F0100216BF03
:1023B00060F3CF329A605A615A69487860F31042EC
:1023C0005A615A69087860F352425A615A69C8786A
:1023D00060F3CB225A615A69087960F3D5425A6199
:1023E0005A69886860F39F525A619A68C96861F3B4
:1023F000D5229A609A6842F480629A60704700BF62
:10240000442F000010B50A4B0A7853F82030586961
:1024100062F3000058614C78586964F34500012A62
:10242000586101BF89785A6961F387125A6110BDFA
:10243000442F0000034B53F82020936843F001031E
:1024400093607047442F0000174B82B053F8203040
:10245000002201925A69162161F345025A619A6875
:1024600042F001029A609A6842F002029A6042F2D7
:102470000F71019A8A4201D9012007E0DA685206F9
:102480000ED59A686FF341029A6000209A686FF344
:1024900000029A605A696FF345025A6102B07047B0
:1024A000019A01320192E4E7442F0000034B53F8F4
:1024B0002020936A43F0010393627047442F000089
:1024C000034B53F82030186AC0F31000704700BF68
:1024D000442F0000044B53F82030DB6823FA01F14D
:1024E00001F00100704700BF4C2F000008B50B4BF6
:1024F00053F820301B6ADB0705D51423084A4343F1
:10250000D3581BB19847BFF34F8F08BD054A52F807
:102510002020D16963F30001D161F4E7642F00004A
:102520006C120020542F000007B50F4B0F4A53F8D0
:10253000203052F82020116A5A6A02F001020192FA
:102540008A0706D50A4A142101FB002042682AB1F5
:102550009047BFF34F8F03B05DF804FBD96962F376
:102560004101D961F5E700BF542F0000642F00003E
:102570006C12002008B50C4B53F820301B6ADB06A8
:1025800006D50A4A142303FB00231B691BB1984795
:10259000BFF34F8F08BD064A52F82020D16963F37C
:1025A0000411D161F4E700BF642F00006C12002019
:1025B000542F000007B50F4B0F4A53F8203052F844
:1025C0002020116ADA6A02F0010201924A0706D558
:1025D0000A4A142101FB002082682AB19047BFF308
:1025E0004F8F03B05DF804FBD96962F38201D961B2
:1025F000F5E700BF542F0000642F00006C1200208C
:1026000007B50F4B0F4A53F8203052F82020116ABB
:102610009A6A02F0010201920A0706D50A4A1421B9
:1026200001FB0020C2682AB19047BFF34F8F03B06F
:102630005DF804FBD96962F3C301D961F5E700BF16
:10264000542F0000642F00006C1200200020FFF7C0
:102650004DBF0020FFF768BF0020FFF78BBF0020B1
:10266000FFF7A8BF0020FFF7CBBF0120FFF73EBF59
:102670000120FFF759BF0120FFF77CBF0120FFF7C2
:1026800099BF0120FFF7BCBF0220FFF72FBF022038
:10269000FFF74ABF0220FFF76DBF0220FFF78ABF96
:1026A0000220FFF7ADBF0320FFF720BF0320FFF795
:1026B0003BBF0320FFF75EBF0320FFF77BBF032074
:1026C000FFF79EBF00292BD0164B53F82030087817
:1026D0001A6860F355521A60DA68888960F30F024D
:1026E000DA604A681868013A62F3144018601A68A0
:1026F000087A60F386121A601A68487A60F3C71283
:102700001A60887A1A6860F309221A6008691A69DF
:1027100060F301021A6149691A6961F311421A6191
:10272000704700BF542F0000034B53F820209368DC
:1027300043F0010393607047542F0000034B53F89C
:1027400020309A6861F311429A607047542F00005C
:10275000024B53F820301966704700BF642F000009
:10276000024B53F82030186E704700BF642F0000F2
:10277000044B53F8203001209B6988401840C84022
:10278000C0B27047642F000008B500218520FEF715
:1027900001FC00218620FEF7FDFB012100220846F6
:1027A000FEF7B0FD0E48FEF76FFB0120FEF77CFD43
:1027B0000220FEF71FFE0320FEF7D6FD0028FAD107
:1027C000A020FEF78BFE0421A020FEF775FCA020C0
:1027D0000421FEF7DFFBBDE80840A020FEF764BE41
:1027E00000100020FEF738BB704700000A4B0B4971
:1027F00000226FF07F401A6008604A601A6842F059
:1028000004021A601A6842F002021A601A6842F062
:1028100001021A60704700BF10E000E014E000E021
:102820000E490F4838B50268D1E9004500686FF0DD
:102830007F439A1A1B1A9A428ABFD1E9004542EA9D
:10284000040043EA040028304FF050024FF0000328
:1028500045F10001FEF758F938BD00BFC012002055
:1028600018E000E008B5FFF7DBFF08BD054930B50B
:10287000D1E9002312F1807443F10005C1E900455C
:1028800030BD00BFC0120020704708B5052164208C
:10289000FEF712FC00216420FEF77CFB6420FEF7AB
:1028A000E9FD6420FEF700FEB420FEF7FDFDC02028
:1028B000FEF7FAFDBDE80840D020FEF7F5BD0000A8
:1028C00038B5FFF7E2FF042205210120FEF76EFE76
:1028D000022200210420FEF769FE022201210420C9
:1028E000FEF764FE022211460420FEF75FFE01227D
:1028F00010460521FEF77CFE012200210420FEF790
:1029000077FE012202210420FEF772FE2E490020EC
:10291000FFF7D8FE00200121FFF710FF0020FFF78E
:1029200003FF01210020FFF723FF0028F9D044F224
:1029300020110020FFF70CFF002403210020FFF7E7
:1029400017FF90B30020FFF70BFF204D28800121D7
:102950000020FFF70DFF0028F9D04FF4434100207D
:10296000FFF7F6FE03210020FFF702FF10B300205F
:10297000FFF7F6FE00232B80154B4FF6FD521A8011
:1029800001210020FFF7F4FE0028F9D04FF4905108
:102990000020FFF7DDFE03210020FFF7E9FE70B104
:1029A0000020FFF7DDFE288038BDB4F5803FFBD066
:1029B0000134C2E7B4F5803FF6D00134D2E7B4F574
:1029C000803FF1D20134E6E7742F0000D2120020DC
:1029D00080090020F8B5042105468820FEF76CFB2D
:1029E00004218C20FEF768FB00218820FEF7D2FA34
:1029F00000218C20FEF7CEFA8820FEF73BFD8C20CC
:102A0000FEF738FD8820FEF74FFD8C20FEF74CFDC9
:102A100000260C272B78F4B2A34200D8F8BD6B68CF
:102A20007C431A19185D5168FFF7B4FC6B68185D98
:102A3000FFF70AFD6B68185DFFF7FCFC0136E9E75C
:102A400073B50E460DF107020DF10601C0B200F09C
:102A500057F8054678BB194B9DF807105C689DF840
:102A6000063003EB430304EB830201EB4101926860
:102A700014F823001144FFF7C5FC9DF8063003EB62
:102A8000430314F82300FFF711FD9DF8063003EB14
:102A90004303072114F82300FFF71CFD0128F4D09D
:102AA0009DF8063003EB430314F82300FFF708FDFD
:102AB000C0F30B003080284602B070BDC42F000068
:102AC00008B5FFF761FEFFF78DFE0948FFF78CFEA2
:102AD0000020FFF78BFE0748FFF7D6FE0648FFF7FA
:102AE000EFFE0648FFF776FF00F02AF8FEE700BF8A
:102AF0008C2F0000942F00009C2F0000C42F00009A
:102B0000032809D8054B00EB4000184443780B70AC
:102B1000837813700020704701207047D82F000081
:102B2000704708B572B60020FFF79CFE62B6002021
:102B3000FFF798FEFFF7F4FFF9E781F308880047F5
:102B40002DE99F484A4B4B4D1B684B494B4A4C4E15
:102B50004C4C01932B60DFF850A1DFF850B10023FB
:102B6000ADF80830ADF80A30ADF80C30ADF80E30E5
:102B70000B7033701370237009278946904600202C
:102B8000FFF770FE404AC830106002A90020FFF72E
:102B900057FF0DF10A010120FFF752FF03A90220A0
:102BA000FFF74EFF0DF10E010320FFF749FFBDF8BF
:102BB00008004EF612314143514534D899F80010BF
:102BC000013189F80010BDF80A00304B43F6DB31C3
:102BD000484398420ED2BDF80C00DFF8D4E04843D9
:102BE000704507D9BDF80E00414399423EBF217898
:102BF000013121700020FFF735FE234A1168401A89
:102C00000028F7DB013F17F0FF07B8D199F8003033
:102C1000042B16D91E4B1B682B602378042B17D965
:102C2000FFF77FFFFEE71B485944814295BF31788B
:102C300098F800100131013194BF317088F800100C
:102C4000C1E73378042B01D9134BE4E7019BE3E799
:102C5000124B134A1B6893420CBF4FF480334FF45E
:102C60008023104A1360D3E90010FFF766FFD9E70D
:102C7000EC2F000004080020C8120020CA12002017
:102C8000C9120020D0120020CC120020C05C150018
:102C9000E42F0000BF29CD02E82F0000FC7F0200D6
:102CA000AA44AA4408ED00E04F7B8900B08476FF77
:102CB0008FBD980000500640045006400850064062
:102CC0000C50064010500640145006401850064064
:102CD0001C50064020500640245006402850064014
:102CE0002C500640305006403450064038500640C4
:102CF0003C50064040500640445006404850064074
:102D00004C50064050500640545006405850064023
:102D10005C500640605006406450064068500640D3
:102D20006C50064070500640745006407850064083
:102D30007C50064080500640845006408850064033
:102D40008C500640905006409450064098500640E3
:102D50009C500640A0500640A4500640A850064093
:102D6000AC500640B0500640B4500640B850064043
:102D7000BC500640C0500640C4500640C8500640F3
:102D8000CC500640D050064000500640045006404B
:102D9000085006400C5006401050064014500640A3
:102DA000185006401C500640205006402450064053
:102DB000285006402C500640305006403450064003
:102DC000385006403C5006404050064044500640B3
:102DD000485006404C500640505006405450064063
:102DE000585006405C500640605006406450064013
:102DF000685006406C5006407050064074500640C3
:102E0000785006407C500640805006408450064072
:102E1000885006408C500640905006409450064022
:102E2000985006409C500640A0500640A4500640D2
:102E3000A8500640AC500640B0500640B450064082
:102E4000B8500640BC500640C0500640C450064032
:102E5000C8500640CC500640D050064000F00F400D
:102E600040F00F4080F00F40C0F00F4000F10F40E5
:102E70000090044000A0044000B004400000054061
:102E8000001005400090044000A0044000B0044041
:102E90000000054000100540040000000200000092
:102EA0000000020000000100000008000000100007
:102EB0000100000020000000400000008000000031
:102EC00000000800000004000000010000000100F4
:102ED0000000020000000000008000000040000030
:102EE0000008000000040000000000400000008016
:102EF00000000004200000004000000080000000EE
:102F000000000800000004000000010000000100B3
:102F100000000200004002400050024000800340D8
:102F20000090034000400440005004400040024034
:102F300000500240008003400090034000400440E5
:102F40000050044000B003400070024000B0034055
:102F50000070024000C0024000D002400000034068
:102F60000010034000C0024000D0024000000340B7
:102F700000100340010000001000000001000000EC
:102F80005E010000020000000200000001000000DD
:102F9000D412002001000000E41200200100000013
:102FA000F812002000010000020000006400000090
:102FB0003F0000000001000002000000640000006B
:102FC0003F000000020000000C1000200007040079
:102FD00002040001040000040000000101000201DD
:102FE000010301020101FEFE0202FDFD0303FCFCE0
:082FF00048DBFF7F0100000037
:102FF8000206000078000000010100000000000047
:10300800A42F0000CC2F000001000000B42F000006
:04301800CF2F0000B6
:020000042000DA
:0408040000000000F0
:02098000000075
:0400000300000511E3
:00000001FF
